:100000002020002023010000210100002101000028
:1000100000000000000000000000000000000000E0
:1000200000000000000000000000000021010000AE
:10003000000000000000000021010000210100007C
:100040002101000021010000210100002101000028
:100050002101000021010000210100002101000018
:100060002101000021010000210100002101000008
:1000700021010000210100002101000021010000F8
:1000800021010000210100002101000021010000E8
:1000900021010000210100002101000021010000D8
:1000A00021010000210100002101000021010000C8
:1000B00010B5074C2378002B07D1064B002B02D03C
:1000C000054800E000BF0123237010BC01BC0047BD
:1000D0000000002000000000F40100000A4B10B5F1
:1000E000002B03D009490A4800E000BF0948036813
:1000F000002B02D110BC01BC0047074B002BF9D0EC
:1001000000F00CF8F6E7C0460000000004000020F4
:10011000F4010000F4010000000000001847C04690
:10012000FEE70F480F4970B5884204D000230E4CFB
:10013000CA18A2420ED300210C4B0D4A93420DD394
:10014000FF210C4B0C4A8B43936000F019F800F030
:1001500015F8FEE7C55804331560E9E702C3EDE77B
:10016000F40100000000002000000020000000203A
:100170001C0000200000000000ED00E0FEE7000091
:1001800070B500260E4D0F4C641BA410A6420BD177
:10019000002600F01FF80C4D0C4C641BA410A64266
:1001A00008D170BC01BC0047B300EB5800F010F858
:1001B0000136EBE7B300EB5800F00AF80136EEE742
:1001C000E0010000E0010000E0010000E4010000A7
:1001D0001847C046F8B5C046F8BC08BC9E467047F4
:1001E000DD000000F8B5C046F8BC08BC9E4670476C
:0401F000B10000005A
:00000001FF
